:1000000000308A00E32800000A108A100A118207D3
:1000100024344734503452344D3443342C34003477
:100020000A108A100A1182072C342C342C344E34D6
:100030002A3425346334253463340D340A340034CF
:10004000523084000008031933280330A100A001B6
:10005000A00B2828A10B27283C30A000A00B2E289D
:100060003128800B252831298316851464008312DA
:1000700085183C28831636280830A000D401A01724
:100080004F28A0134F280310851C0314D40C2017ED
:100090004F282013A00B43285408A1005B28A73049
:1000A000A01B2D30A100A10B53280000A01B41284C
:1000B000201B4928432800343530D200D30153088F
:1000C000053C031C6A282530530784000008D2062B
:1000D000D30A5F282B08D206D3015308073C031C20
:1000E00078282C30530784000008D206D30A6D28E4
:1000F000D3015308073C031C842834305307840081
:100100000008D206D30A7928D3015308033C031C04
:1001100090283C30530784000008D206D30A852873
:10012000D3015308053C031C9C284230530784002C
:100130000008D206D30A9128D3015308053C031CBA
:10014000A8284830530784000008D206D30A9D2807
:10015000520EA0000F30A0052008303ECE005208FD
:100160000F39303ECF004E08393C0318B92807300C
:10017000CE074F08393C0318BF280730CF07F229B4
:1001800083160512831205160830A100C728000047
:10019000A117D828A113D30C03180512031C0516A8
:1001A0002117D8282113A10BCB28D628000005122F
:1001B000A7308400840BDA2800006400A11BCA2841
:1001C000211BD228003484011F30830583160512B9
:1001D000831205121F1383161F109F101F119F11EA
:1001E0000730831299003030BC00BD01BE01BF0151
:1001F000C001C101C200C301C401C501C601C701DC
:100200001F1383161F109F101F119F1183121F10A1
:1002100083160108C739083881000F308312A00007
:1002200007308101813084000008F03907388000F0
:1002300064000008F739A019F0392004800090010B
:10024000073099008316050808308312A000A00B20
:10025000272919088C11831699010A308312D200BC
:10026000202864003030BE00BF00C000C200C300C0
:10027000C400C500C60034202108243C03194229CB
:1002800064003B2934202108473C031D31293420D8
:100290002108503C031D312934202108523C031D04
:1002A0003129342021084D3C031D312934202108F7
:1002B000433C031D31293420D0015008053C031C68
:1002C0006C29253050078400D30034205308840063
:1002D00021088000D00A5D29342021082C3C031D10
:1002E0006C2934202108AB00342034202108AC00D4
:1002F00034202108AD0034202108AE00342021082C
:10030000AF00342034202108B00034202108B1008F
:1003100034202108B2003420342034202108B300D6
:100320003420342034202108B40034202108B500C2
:1003300034202108B60034202108B70034203420AE
:100340002108B80034202108B90034202108BA005F
:100350003420342034202108BB003420D001500840
:10036000053C031CC12934202108D10051082C3C34
:100370000319C1295008D00A3C3E8400510880006E
:10038000AF29D0015008053C031CD4293420210892
:10039000D10051082C3C0319D4295008D00A423E00
:1003A000840051088000C22934202108C800480870
:1003B0002C3C031DDF2934202108C800D729013037
:1003C000D0005008053C031CF02948305007840039
:1003D000D30034205308840021088000D00AE1298A
:1003E00064005C28D20152080420D20AA000D30085
:1003F000C02007305202031DF329D0015008053CEC
:10040000031C0B2A2530500784000008D200D300BB
:10041000C020D00AFE292C30D300C0202B08D300E6
:10042000C0202C30D300C0202C08D300C0202D08C1
:10043000D300C0202E08D300C0202F08D300C02036
:100440002E30D300C0203008D300C0203108D300A4
:10045000C0203208D300C0202C30D300C020330885
:10046000D300C0202C30D300C0203030D300C020B7
:100470003408D300C0203508D300C0203608D3008C
:10048000C0203708D300C0202E30D300C020380849
:10049000D300C0203908D300C0203A08D300C020C0
:1004A0002C30D300C0203B08D300C0202C30D30018
:1004B000C020D0015008033C031C672A3C30500781
:1004C00084000008D200D300C020D00A5A2A2C3061
:1004D000D300C020D0015008053C031C782A4230CC
:1004E000500784000008D200D300C020D00A6B2A35
:1004F0002C30D300C020D0015008053C031C892AB1
:100500004830500784000008D200D300C020D00A31
:100510007C2AD20152081020D20AA000D300C020A9
:1005200005305202031D8A2A4E08D300C0204F080E
:10053000D300C0200D30D300C0200A30D300C0202B
:0405400031296300FA
:02400E008B31F4
:00000001FF
